:1000000000308A00862900000A108A100A1182072F
:1000100028340C34013406340A108A100A1182077D
:100020007334743461347434753473343A34203432
:100030002534583400348316061183120615280817
:100040009300831614182628831221288312003463
:1000500031308400000803193C280130F800F70112
:10006000F70B3028F80B2F284A30F700F70B36280B
:1000700000000000800B2D2800340508F039B8007E
:1000800037080F393804850006148316061000005F
:10009000831206108316061083120034B508031D60
:1000A0005328861154288615831686118312B60E9E
:1000B0003608B7003D20B60E3608B7003D200D309B
:1000C000F700F70B612800341430B1002820F0301D
:1000D00083168505831286118316861183120610F6
:1000E000831606108312A8012808023C031C8028EE
:1000F0000230B10028200330B7003D20A80A742840
:100100000D30F700F70B82280230B7003D200D308C
:10011000F700F70B8928A8012808023C031C9C283B
:1001200028080420A900B5012908B6004E20023095
:10013000B1002820A80A8C288A11D4290130310264
:10014000B3003208023C031DA7284030B307330830
:100150008038B400B5013408B6004E2000343008B1
:100160000C3A0319BD28063A0319C528073A0319A2
:10017000CB28053A0319D028D528B5010130B6009F
:100180004E200230B1002820E1280130B1000230B9
:10019000B2009E20E1280130B100B2009E20E1288B
:1001A000B5011030B6004E20E12830081F3C031C7A
:1001B000DB280730B0050130B5003008B6004E200E
:1001C000E1280034AA1BF4280F30F700290EF705A8
:1001D0000A3077020318EF283030F707F1282A0891
:1001E000F7077708B000AF200F30A9050A302902C1
:1001F0000318FC283030FE28AA132A08A90729086A
:10020000B000AF208A11EB290408AF00A91F112903
:100210002D30B000AF208403A809A909A80A03194A
:10022000A90A290EF038AB00AB07E23EAC00323E23
:10023000AE0029080F39AC07AC07AE07E93EAD00A8
:10024000AD07AD07280E0F39AD07AE07AD0DAE0DEA
:10025000AE09AE0D28080F39AE07AB0D0730AA0066
:100260000A30AE07AD03031C3129AD07AC03031CF4
:100270003529AC07AB03031C3929AB07AA03031CC0
:100280003D292A30840007302F0584072E300402D0
:10029000031966290008F700031D54292F1A642941
:1002A000AF195629203057290830AF003030F707F2
:1002B000A9010408A8007708AA007708B000AF20B9
:1002C000280884002A08F700840A46290008F70055
:1002D0003030F7077708B000AF20003483160611DE
:1002E000831206152808930083161418792983129F
:1002F0007429061583121308930183161418822992
:1003000083127D2983121308F800003484011F3002
:10031000830583161F129F121B0880399B0007302C
:100320009C001C0883120D13603083168F0083120B
:10033000A201A301A401A50183161F129F121B088D
:1003400080399B0083121F109412831606118614A5
:100350000612323083129400003083169400010894
:10036000C73908388100831290010030F8009200EC
:1003700000308316920007309C0005080330F70018
:10038000F70BC0291C0883120D1383169D018530BD
:100390008312A8001B20A8011B208630A8001B2068
:1003A0000630A8001B206428C830B1002820013086
:1003B000B100B2009E20A80128080C20A80AF7006E
:1003C000B000AF2008302802031DDC292108A90055
:1003D0003730AA00E2281430B10028200130B100E3
:1003E0000230B2009E205830B000AF203D30B00047
:1003F000AF20103084002308A9002208A80004219F
:100400002030B000AF205930B000AF203D30B000F8
:10041000AF20103084002508A9002408A80004217A
:100420001430B10028200230A8006E217808A10005
:100430000330A8006E217808A6000430A8006E21C1
:100440007808A700FA012608A61BFA03A2070318DA
:10045000A30A7A08A307FA012708A71BFA03A4072F
:0C0460000318A50A7A08A507D729630035
:04400E00793FFF3FB8
:00000001FF
